S1048000007B
S123C000C783C765C78CC7C0C76BC773C77BC7CEC7E6C7DEC7EEC840C836C82AC82FC84982
S123C020C861C8AFC871C881C891C937C957C963C977C789CA5AC98DC9A2C997CAB6CAC254
S123C040CACDC9BFC9ABC9C9C9D3C9E3CA24CA50CA5FCA7BCA8ACA99CA30CA40CA15C9FB9B
S123C060CAE2CAE6CAECCAFDCB10CB03CB46CB18CB56CBB9CBCECBDCCBEECB91CB9BCB74A7
S123C080CBA4D7CAD776D7A0D7B8D7DDD7F0D802D80DD825D84AD85AD7FBD875D889D894C2
S123C0A0D86AD89FD8AAD8B5D8C7D8D5D8E3D785D90BD930D91BD8F1DD3EDE1CDE20DE6551
S111C0C0DADECBA7CBB0DAB7DAEDDAFE000099
S123C500FCFF0227358E00FFBDE11B1AB3FF022608CC0000FDFF022021BDDBD2CEC52DBD8A
S123C520DD2DB67F0084C088C027F720134D454D4F5259204641554C54008EFEFF7F003C20
S123C5408D352016B67F0084038103260D8E00FF0FBDE11BFDFF027EE0B7B67F0027037E27
S123C560C70EB680004A26F7CC8001CEC300ED008600A7097EC70ECE002A4FA700088C006F
S123C5803926F8CE1000860AB77F00970E86FF9722972397249725CC07C0DD261C39801D00
S123C5A0282086B0A72B860CA72D86079739BDDBD2CC0000DD0CDD12DD148608970BCCC1A8
S123C5C010DD16DD18DD1A8620B7C6F4CEC300C6208640A7098FC300108F5A26F6CEC3006C
S123C5E0DF08CCC200ED00CCFE00ED04C30001ED02830100ED06860AA7088620A709EF0C60
S123C600EF0EDC0CC30001DD0CED0ABDDAFECEC635A6002706BDDBA40820F6CE10001C20E8
S123C6200118CE3000180926FC1D20011D0008CC0000DD263946696E67657220426F617232
S123C640642020202076322E38332031312F32342F39380A008D6B8D74816125F8817326DE
S123C66004863E2068368D513C18388D4C328172270D8177270F816327118162271B39A646
S123C680008D4A2010188FE700200A188FA400A700EA00E700863E2034188F373C32331B62
S123C6A0331B97015D270C8D19A7009B019701085A26F496018D1620DC8D07368D0416322A
S123C6C08F39B6102E842027F9B6102F39F6102EC48027F9B7102F39DE08A608970A1AEEA4
S123C6E000EE0218E600F7C6ED1808FCC000FDC6F2BDFFFF20ED8620B7C6F4DC088FED02CC
S123C7001AEF00A60981402604EE0CDF0839963C260CCE10001F2E2005BDC65520F0120BFF
S123C72002ECDE08EE0EDF088CC3002607DC1EC30001DD1EA609810026D4BDC6D8810027DC
S123C740CD814027C9812027048602200286048D0220BB9701940B910126013996019A0B88
S123C760970B7EC6CDEC02A300201CEC02A400E4012014EC02AA00EA01200CEC02A800E85D
S123C780012004EC00E302ED020808398D26A601E6033DDD00A600E6033DDB00D700EC019F
S123C7A03DDB00D7007D000727064F5F930020D7DC0020D37F00078D6308088D5F09093911
S123C7C0BDC7B4EC023CEE0002DF003820D7EC00A3022705CC000020AECC000120A9EC021A
S123C7E0A3002EF520EEEC02A3002DED20E63CEC002B1C26043808083937368605B7C8031C
S123C800EC02380027030926FA380808ED00394F5FA30037368604B7C80320E46D002A09BF
S123C8204F5FA300ED007300073963006301394F5FA300ED0039EC002705CC0001ED003981
S123C840EC0027F64F5FED0039EC02E306DD00E601E905A600A904ED04DC00ED06C6043A57
S123C86039EC06A302DD00E605E201A604A20020E6EC06A302E605E201A604A2002D1E20CB
S123C88025EC02A306E601E205A600A2042D0E2015EC06A302260FEC04A3002609C6063ABA
S123C8A0CC0001ED0039C6063ACC0000ED00397F0007BDC94D3CC6043ABDC94DCE0000DF70
S123C8C00038A603E6073DDD02A603E6063DD301DD01960089009700A602E6073DD301DDAD
S123C8E001960089009700A603E6053DD300DD00A602E6063DD300DD00A601E6073DD300D7
S123C900DD00EC033DDB00D700A602E6053DDB00D700A601E6063DDB00D700A600E6073D84
S123C920DB00D700C6043ADC02ED02DC00ED007D000727028D0139CC0000A302DD00C6001F
S123C940E2018600A200ED00DC00ED02396D002A058DE47300073918EC00180818080909C1
S123C960ED003918EC020909ED0018EC00180818081808180820E718E600183A18A60009E6
S123C980A70018095A26F518E600183A393CCDEE00E600384F20C38FCDEE00EE028F0909AB
S123C9A0ED008FCDEE00EE008F20AF18E6003C3AEC00DD00EC02380909ED00DC00209D18DD
S123C9C0E6003C3AEC003820933CA601CDEE00A70020083CEC00CDEE00ED0018083818086B
S123C9E00808393CEC00DD00EC02CDEE00ED02DC00ED0038C6043A57183A39EC00DD00ECB1
S123CA0002D70718E6003C3AD607ED02DC00ED0038080820C9EC00D70118E6003C3AD601E9
S123CA20ED0020B9A6013CEE02273FA70038202AA601B7CA3C3CEE0227301C00FF38201A56
S123CA40A601B7CA4C3CEE0227201D00FF38200AEC003CEE022713ED00380808080839ECB1
S123CA6000DD00EC023CEE0426063886057EDE71ED02DC00ED0038080820DFEC003CEE02E6
S123CA8027E8E70038ED02080839EC003CEE0227D9ED0038ED02080839EC00DD00EC023CC4
S123CAA0EE0427C6ED02DC00ED0038EC02ED04DC00ED020808393CEE0027AFE6004F38ED56
S123CAC000393CEE0027A3EC0038ED00393CEE002798EC00DD00EC02380909ED02DC00ED39
S123CAE0003918EE00391AEE00080839EC00260618EE0008083918081808080839EC002667
S123CB00EF20F3EC0027EFCC0001ED0018EE0039EC0026E218EE0039EC00DD0018EC00DF35
S123CB2004D3048F1AEE002705DC00ED0039DE088640A7098621B7C6F4EC0C1AEE0E8FCD73
S123CB40EF0C1AEF0E3918EC00DF00D3008F1AEE0027DB080839EC00DD00EC02DD0218EC54
S123CB6000DF04D3048F1AEE0227C3DC00ED00DC02ED0239DF00DE08DC00A306CDA30025C6
S123CB800718081808DE00391809DE0086047EDE718F18E3008F18081808393C323318E3AF
S123CBA0007EC95AEE0039EC00DD3A0808180839DC3A0909ED00180839EC003CEE021AA3FA
S123CBC000382427E302C30002ED02080839EC003CEE021AA3003824120520E8EC003CEE86
S123CBE0021AA300382404050520D97EDE6BEC003CEE021AA3003824F218A60018083D20EA
S123CC00C33CBDD6E6CE00003CDF41DF437F00451830CDEE06A600BDCD592528812D260BCA
S123CC2073004508A600BDCD592519812E260B08A600BDCD5924037ECCC73131BDD6F038A3
S123CC40860F0D39A600BDCD592477BDCCD80824F37C0041A60008BDCD5925F5812E260A0A
S123CC60A600BDCD5924030820F681452707816527037ECD1B08A600BDCD592515812D27D8
S123CC8006812B270520B318630008A600BDCD5924A8803018A70108A600BDCD59241418B6
S123CCA0E601585818EB015880301B18A701088126228718A601186D002A01409B41974137
S123CCC02059812E26A408A600BDCD59249C8D0808258D7A004120EF96429747DC43DD48FA
S123CCE005790042252C057900422526D3483696429947974232251A05790042DD432512AA
S123CD00E600C0304FD343DD43964289002503974239DC48DD439647974239CDEF06CE0056
S123CD2041BDCD84272C964118A70186969741BDCD65186D01271B2A0BCECD8FBDD71918E7
S123CD4060012006CECD93BDD719BDCDA3186A0126F83131BDD6F038398130250681392291
S123CD60020D390C39CE00418D1A27147D00422B0FDC437A0041270A057900422AF5DD432E
S123CD800C390D393736EC002602EC023233393DCCCCCD41200000BDD03FBDD6E6BDCF0E15
S123CDA0BDD6F07D004127057D0046260ACC00009745DD41DD43399645984A974596419BE5
S123CDC0462A0924168606CEFFFF2009250D8607CE0000DF44DF41DF430D398B829741CE30
S123CDE000003C3C30BDCE1C6D002B0B69036902690169007A00416D032A13A6024CA7028E
S123CE00260CC601E3002404467C0041ED0038DF42329744317D004127B45F399649D64459
S123CE203DA7019648D6443DE300ED009649D6433DE300A70324026C026F006F019647D61C
S123CE40443DE302ED029648D6433DE302ED0224026C019649D6423DE302ED0224026C0143
S123CE609647D6433DE301ED0124026C009648D6423DE301ED0124026C009647D6423DE36B
S123CE8000ED0039BDD6E6CED412BDD7197D0045270373004ABDCF40BDD6F04FD641C17FF0
S123CEA024035F201B53C3FF902F178FDC422001040926FC7D00452A074353C300012A024C
S123CEC00C3986090D39CC0000DD004FD641C17F24035F203353C3FFA02F2F8F96445FDD54
S123CEE000DC422007047600007600010926F67D00452A147300007300014353DE0008DF91
S123CF00002605C300012A020C3986090D39BDD37ACE0049964680972A1BC6038B082A09F0
S123CF206F00095A26F66F0039C6804A2B035720FAE400E7008D028D07964A88FF974A39B9
S123CF409641260EDC46DD41DC48DD43964A97455F397D004627F9D645D84A90462510813E
S123CF601822ED183C36CE004718CE0042201740811822D0183C3696469741964A9745CEF5
S123CF80004218CE004717363636A8003617A8013617A8023630A606E7061684074CC41808
S123CFA05454543AE6034A27095666026601660020F45618A602A900974418A601A901979B
S123CFC04318A600A902974230A6062B15245A7600427600437600447C0041264CCCCDC576
S123CFE02053251B73004570004424087C004326037C004270004324037C00427000427D75
S123D00000422B2526139641800823269741DC4327207F0044DD4220E67A00412714780005
S123D020447900437900422AF01AEE07C6093A355F39CCCDCE1AEE07ED07C6073A3539CE85
S123D0400046BDCD84260486080D39CE0041BDCD8426020C39BDD6E6964A98459745CE0010
S123D060003C3C3C86183630DC421A934726049644914924107C0046261986060D3838388E
S123D08031BDD6F039DC439348DD439642924797426A007400477600487600499641D64666
S123D0A0501B2B062506860720D325CE8B7F9741DC42ED049644A706DC439348DD439642C8
S123D0C0924797422A08EC04DD42A60697446903690269017800447900437900426A0026CE
S123D0E0CF630163026303DC43934896429247EC0224030C2003C30001DD43A60189009794
S123D1004224117600427600437600447C004126037ED07A0C7ED07D3CCE0041BDCD842665
S123D1200738CC3000ED0039DE413CDE433C964536BDD6E6CE00003C3C3C1830CDEE0F862E
S123D140207D004527057F0045862DA70008CDEF00CED282BDD719BDD2862E19CED27EBDD5
S123D160D719BDD2862E16186A02CECD93BDD719BDCDA320DC186C02CECD8F20F0CED41266
S123D180BDD719BDCF40D641C07F50CB17200A7400427600437600445A26F4860118A7037A
S123D1A018A6028B082B0A810824064A18A7038602800218A702186D032E15862ECDEE001F
S123D1C0A70008186D0327058630A70008CDEF00CED269860718A705186F04DC43A301DD42
S123D1E0439642A20097422505186C0420EDDC43E301DD439642A900974218A6048B303CA0
S123D200CDEE00A70008186A032605862EA70008CDEF0038080808186A0526BCCDEE000954
S123D220A600813027F90818E602272A8645A70008862BA7005D2A0550862DA70008CDEF4E
S123D240004FCE000A02378FCB30CDEE00E7000833CB30E700086F00383838BDD6F03297B6
S123D2604538DF4338DF4138390F42400186A00027100003E800006400000A00000149743C
S123D28023FE4B18967F964A2A12D6452A0EDC461A93412617DC481A934320109145260CE9
S123D2A0DC411A93462605DC431A93480784F424028A080639CE008EC3000026057ECDCE42
S123D2C009052AFCDD427F00448F9745D7415F394D2AE24353C30001CEFF8E20DBCE009EA4
S123D2E0C30000261118DE0026037ECDCE0978000179000059492AF5DD42960097448F9786
S123D30045D7415F394D2AD57300007300014353DE0008DF002603C30001CEFF9E20C1CE7F
S123D3200041BDCD842601397D00452A04860A0D39BDD6E6860436DE433CDE413C18308DAE
S123D340399646807E4C2A03442003448B7E9746BDD03FBDCF407A00418D1F18EC00DD418B
S123D36018EC02DD43186A0426E6DC46DD41DC48DD43383831BDD6F05F39DC41DD46DC4352
S123D380DD489645974A39BDD6E6CED4E1BDD719BDD03FBDD6F0DC411A8385B32B0B7D00D2
S123D3A04526037ECDC57ECDCEBDD6E69645367F0045BDCF0EDC4627068086544C26FC5C77
S123D3C037CED3F6BDD6A6CED3F2BDD7192003BDCDA3306A0026F832324D2A0CBDD37ACE3B
S123D3E0D63ABDD700BDD03FBDD6F05F39BDD6E620EA402DF8543638EF1D37D00D0139504A
S123D4000D013AB60B613C0888893D2AAAAB3E2AAAAB3F0000003F8000003F800000FFBD57
S123D420D43BBDCDA37ED3968D11BDD6E6CED4E1BDD719BDCDA3BDD6F05F399645270486AA
S123D4400C0D39964127F8BDD6E63C3C30BDD7314FD641C07F2A0143BDD2D0CED4DDBDD715
S123D46019BDCDA330BDD719BDD731867F97463C3C30BDD73FCED63ABDD700BDCF4030BD38
S123D480D719BDD731CED4D9BDD700BDCF4030BDD719BDD03F30BDD731BDD37ABDCDA3CE55
S123D4A0D4BCBDD6A630BDD719BDCDA3383830BDD719BDCF403838BDD6F05F393E1D89D934
S123D4C03E3A2E8C3E638E393E9249253ECCCCCD3F2AAAAB40000000FFBF8000003F3172AF
S123D4E0183EDE5BD9860E0D39860D0D39BDD6E69645367F0045CED63ABDD719BDD2862FF0
S123D50007BDD3ED86FF20014F363C3C30BDD731BDD37ABDCDA3CED544BDD6A630BDD719B7
S123D520BDCDA33838324D270CCED540BDD719730045BDCF40BDD690329745BDD6F05F3938
S123D5403FC90FDBBCE2DD1B3D70F0F1BD8888893D9D89D9BDBA2E8C3DE38E39BE124925C9
S123D5603E4CCCCDBEAAAAAB3F800000FFBDD6E64F2005BDD6E686F036CED658BDD719202E
S123D58003BDCF40964526F92003BDCF35BDD2862EF88D61240930A6002B04880FA7008DB4
S123D5A054240930A6002A04880FA7008D47240730A60088F0A700CED69EBDD719BDCDA394
S123D5C0BDD37ABDCDA33C3C30BDD73FA6042A05CED63F2003CED62ABDD6A630A60447246A
S123D5E0037300454D2B06BDD719BDCDA3383831BDD6F05F397A0046BDD2862E020C397C92
S123D6000046730045BDCF407A00460D39BDCF0EDC41DE46DD46DF41DC43DE48DD48DF438C
S123D6209645D64A974AD7455F393638EF1DB9500D013C088889BE2AAAAB3F800000FF373E
S123D640D00D01BAB60B613D2AAAABBF0000003F800000FF40490FDB43B40000BDD6E6BD33
S123D660D37ABDD573BDD610BDD56DBDD03F2407BDD6F0860B0D39BDD6F05F397FFFFFFFCA
S123D680BDD6E6CED69EBDD719BDCDA3BDD6F039BDD6E6CED6A220EECED6547ED7003C8E51
S123D6A0FA3142652EE18FDE413CDE433C8F9645363CCC0000DD41DD43DD44201030A6022F
S123D6C0974AEC03DD48EC05DD46BDCDA330EE00BDD719BDCF4038C6043A3CA6004326DD15
S123D6E030C6073A3539383C3C8F3037367ED73F300808BDD71938313131316E00CED63ADC
S123D7007F0045EC02DD43EC00052403730045974127020D56D7425F397F004AEC02DD4872
S123D720EC0005240373004A974627020D56D74739DC43ED02DC4158D1454656ED0039DC19
S123D74048ED02DC4658D14A4656ED00397F00455F397D00422705CC7F80DD414F5FDD4339
S123D760397D004227037300455F39BDD71908080808BDD700393C183CEC00BDD2D018386E
S123D78038090920AC3C183C0808BDD7000909EE00BDD118183838EC00ED040808080839D7
S123D7A03C183CBDD700BDCEC618383824037EDE71ED00DC00ED02393C183CEC02DD00EC3C
S123D7C000BDD3051838387ED7313C183CBDD700BDCE9B18383824037EDE71205D3C183CCF
S123D7E0BDD76BBDCF40183838080808087ED7313C183CBDD76BBDCF3520EBA6008880A77C
S123D80000393C183CBDD76BBDCDA320093C183CBDD76BBDD03F18383824037EDE710808FF
S123D82008087ED7313C183CBDD76BBDD286183838260CCC0001080808080808ED003908C5
S123D84008080808086F006F01393C183CBDD76BBDD2861838382BDB20E53C183CBDD76BBE
S123D860BDD2861838382ECB20D53C183CBDD76BBDD41F20A13C183CBDD700BDD31F1838F6
S123D8803824037EDE717ED7313C183CBDD700BDD39620EA3C183CBDD700BDD38720DF3C08
S123D8A0183CBDD700BDD43B20D43C183CBDD700BDD42820C93C183CBDD700BDD4ED073617
S123D8C0BDD680320620B73C183CBDD700BDD690BDD56D20A93C183CBDD700BDD690BDD53A
S123D8E073209B3C183CBDD700BDD690BDD65C208D8602E6019D4B080839BDDBEAA600BD8E
S123D900DCCAA601BDDCCA08082003BDDBEAA600BDDCCAA601BDDCCA080839BDDBEA3CEE96
S123D920008602E60027059D4B0820F738080839183CDF00BDDB4A1A830051240C8621B730
S123D940C6F4DE001838180939DE00DC00C30002E300DD02830002DD04DE02EE000808A656
S123D9600026037EDAA5812527037EDA9308A6008166261BDF02DE0409093CBDD700380906
S123D98009DF04CEC100BDD118CEC1007EDA858164267DDF0218CEC100DE040909DF04EC23
S123D9A0022A0C862D18A7001808CC0000A302CE000A02378FCE000A02378FCE000A0237D7
S123D9C08FCE000A02378FCE000A0237183C388601335D27064FCB30E70008334D27045DF2
S123D9E027064FCB30E70008334D27045D27064FCB30E70008334D27045D27064FCB30E7E9
S123DA00000833CB30E700085FE700CEC10020758178262ADF02DE040909DF04A602BDDC31
S123DA20B0BDDB92257217BDDB92256CA603BDDCB0BDDB92256217BDDB92255C20618163D5
S123DA402611DF02DE040909DF04A603BDDB922547204C8162261EDF02DE040909DF04E663
S123DA600318CE00085886308900BDDB922529180926F2202A8173261ADF02DE040909DF37
S123DA8004EE020808A6002708BDDB92250A0820F4200CBDDB922409860ABDDBA42006DEE1
S123DAA002087ED95FDE00DC00C30002E3008FCC0000ED001838393CDC14C300011A9314BE
S123DAC026FBC30001CE0000081A931426FA8F380909ED00CC000C0909ED007EC78C090926
S123DAE009090FDC14ED02DC120EED0039EC0008083C183CEE00AD00183838ED00390F3CE0
S123DB00183CB6103C84402605CEFF002003CEBF003CC6C03A18CEE12D1AEF0008083C32C8
S123DB20324D26F538CCC500EDFECCDEEBEDE2CCDEDEEDE0CE10006F226F248600A7211C6E
S123DB4023181C22181838380E39960B84082707CC00F0DD062016DC1893162307830001E6
S123DB60DD062009CC00F09316D318DD06960B84102705CC00F02012DC1A931623058300C9
S123DB80012007CC00F09316D31A1A93062302DC06393736BDDB4A1A83000224040D32338C
S123DBA039322001370F3CDE16088CC2002603CEC110DF16A700960B840827119C18260D59
S123DBC0DE18088CC2002603CEC110DF1838330C0E398D79CC00389D4BC60C9D4B8D1986A0
S123DBE001970F8608971C4F971DCC00019D4BC6069D4BC68F9D4B39CC00409D4B8602CE0D
S123DC00DC0DE6009D4B088CDC4D26F639000A1F1F0E04000000001111110F010E0000008C
S123DC2000000C040800000F11110F010E00000C0C000C0C0000000C0C000C040802000611
S123DC40020202120C00000A0E04000000CEDC6218CE004BA60018A7000818088CDCB02678
S123DC60F339FF0096CE10000F1D3C201D0010B700986F078104260F8601B710041C00104F
S123DC80A6031D0010201E8601B710041C0010A6031D001086FFA707B60098A704E7031CE6
S123DCA000101D00101C3C20FE00960E3900000036840F8B30813A2B028B071632444444BE
S123DCC0448B30813A2B028B0739BDDCB0371686029D4B339D4B39CE000A02378FCE000ABC
S123DCE002378FCE000A02378FCE000A02378FCE000A02379D4BCC00019D4BCC00079D4BAF
S123DD00CC008F9D4B860233CB309D4B33CB309D4BC62E9D4B33CB309D4B33CB309D4B33CD
S123DD20CB309D4BC66D9D4BC6739D4B39CC00029D4B8602E60027059D4B0820F739183CA3
S123DD40DF00CC7FFFDD04CEC3001AEE0E188CC3002607CCE400DD06200518EC04DD06ECEB
S123DD600693063CDE00A300382B091A93042E04DF02DD04188CC3002705183C3820CBDC4C
S123DD80041A837FFF260486012015CEC310A609814027158FC300108F8C620026F08602B0
S123DDA0DE00183818097EDE713C1838DE02EE0E1AEF0CCDEF0EDE021AEF0ECDEF0CEC064B
S123DDC083000118ED04C30001DE00A30018ED06A60318A708EC0418ED00860018A709DCD3
S123DDE00CC30001DD0C18ED0ADC00E306C30008EE068F09DF0018DF0218EE0436A6001865
S123DE00A7003209180983000126F1DE0218081AEF02DE0009DC0CED0018383986202051F9
S123DE203CEC00DD00CEC300EC0A1A9300270EEE0E8CC30026F238CC0001ED00399C082618
S123DE4004387ECB2E183C8640A7098621B7C6F4EC0C1AEE0E8FCDEF0C1AEF0E183838CC59
S123DE600000ED00398621B7C6F4391809860320003CDE084D2602861FA70997018621B77B
S123DE80C6F4960181202431CEDEBBA6002708BDDB9225F70820F44FD601C00A25034C2015
S123DEA0F9CB0A8B30BDDB9225FB178B30BDDB9225FB860ABDDB9225FB38390A52554E54D1
S123DEC0494D45204552522000CE1000DC28E316ED161D237FB610008880B710003BCE10EF
S123DEE000DC26E31EED1E1D23F73BCE1000CC07D0E31CED1C1D23EFA622368408A7220E85
S123DF00DE1408DF142605DE1208DF127A000A26058621B7C6F486049D4B848027037EDF38
S123DF20F89615843F2640960F8101223A0F4FC6CF9D4BDC1E1A8300642D0BCC0000DD1EB9
S123DF40961C880C971C961C84082704C6002002C60786029D4B4FD611C1102502CB30CA43
S123DF60809D4B0E7EDFF89639840126037EDFF8960F8102245EDE1A9C16277C088CC200B3
S123DF802603CEC110DF1AE600960F81002634C10A26068601970F205F9611811F27594CA0
S123DFA09711811126074F37C6C09D4B33C120250CC17F2208CEE03AC0203AE60086029D46
S123DFC04B20358101260DD710FCE0289D4B8602970F2024810A2712CEE028D60F3AEC00FE
S123DFE09D4B960F8B02970F200E8600970F86019711D610C10A26B5D60E963984042720C6
S123E000C6FF96229B3D973D5696239B3E973E5696249B3F973F5696259B40974056D40E5B
S123E020F77F0032B710223B0001000600CF020000020011495557777FFF2021222324256C
S123E040262728292A2B022D2E2F3031323334353637383904053C3D3E3F404142434445A2
S123E060464748494A4B4C4D4E4F505152535455565758595A5B5C5D5E5F606162636465EC
S123E08066036869066B6C6D6E6FF0F172737475767778017A7B7C7D7E7F18CE03E8180929
S123E0A026FCCE10001F000433CC1BE61F00042C83000126F7203937368D56CC00029D4BEA
S123E0C0CEE0E58602E60027059D4B0820F732BDDCCA32BDDCCA8602C6299D4BCE10001C85
S123E0E028204F06CF2A48616C7465642A2028008D1FCEE101BDDD2DCE10001D23FB8D16E3
S123E1003B2D504F57455220474C495443482D20008601979439860E979439CE80004F5FFF
S111E120E3008FC300028F8CFF0226F4393B0C
S123BFC0E12DE12DE12DE12DE12DE12DE12DE12DE12DE12DE12DE12DE12DE12DE12DE12D7D
S123BFE0DEDEDEEBE12DE12DE12DE12DE12DE09AE12DE12DE12DE12DE12DE12DE12DC500D1
S123FFC0E12DE12DE12DE12DE12DE12DE12DE12DE12DE12DE12DE12DE12DE12DE12DE12D3D
S123FFE0DEDEDEEBE12DE12DE12DE12DE12DE09AE12DE12DE12DE12DE12DE12DE12DC50091
S105FF020000F9
S105FF000253A6
S9030000FC
